:03000000021642A3
:0C164200787FE4F6D8FD75816E021689F1
:101CD900AE071FEE600DE4FCFD0DED70010C4C60CC
:031CE900EF80F693
:011CEC0022D5
:0D1DC000E4F5C7F5C5F5C675C380F5C4226E
:101CAC0075C78175C5018FC48EC375C65A75C6A517
:061CBC0000AFC2121DC0C2
:011CC20022FF
:101CC30075C78175C5028FC48EC38DC275C65A751B
:061CD300C6A500021DC0C1
:101CED0075C78175C5038FC48EC375C65A75C6A5D4
:041CFD0000021DC004
:0611F400016D01016E0116
:051A7900E5124480FFAE
:021A7E008F13C4
:101A8000E4F514E51330E011D2C0121DD9121DD9AE
:101A9000C2C07F02121D72800FD2C07F02121D725F
:101AA000C2C0121DD9121DD9E513C313F5130514B5
:071AB000E514C3940840CCCB
:011AB700220C
:101B2D008F12D2C0121DA3C2C0121DF0121DF012D1
:101B3D001DF0AF12121A7E121DF0121DF0121DF0C3
:101B4D00AF12121A7E121DF0121DF0121DF0AF12FF
:091B5D00121A7E121DB2021E04D0
:101A31008F12D2231512D2C0121DA3C2C0121DCD06
:101A4100121A79121DCD121A79121DCD121A79129C
:101A51001DB2121DCD121DCD7F90121A7E121DCD09
:101A61007F90121A7E121DCD7F90121A7E121DB226
:081A7100121DCDC2B7C2B6225E
:0F1D940030230BC2237FA0121B2DD2B7D2B62251
:101D0100EF64096003BF0A027F08C374099F44A0FE
:041D1100FF021B2D85
:1011FA00C121016800016C00C12002690000016B75
:01120A0002E1
:03000B00020841A7
:10084100C0E0C0F0C083C082C0D075D008758A9A5C
:10085100758CA9300F0AE528600415288002C20FA3
:100861000568056CE56CC394144003756C00E5687C
:10087100C394055003020A5575680030001BE54E0C
:100881007017E537153770021536D3E5379400E553
:100891003694005004C200C2A330203BE56A45698A
:1008A100600AE56A156A702F1569802BC220E54E32
:1008B10064036023E54E6404601DE54E6405601722
:1008C100E54E64066011E54E640D600B201108E5EC
:1008D1004E64136002D2B6E55DB40113E560455F75
:1008E100600AE56015607007155F8003755D023071
:1008F1001016E5454544600AE5451545700A15445D
:100901008006C210D2C2D29130174DE54D454C60E0
:100911000AE54D154D7041154C803DC217C202C20A
:1009210019C206C216753400754E00C211D2C4D266
:1009310021C2A6D2C5D2C1C287C28575250175263D
:1009410090D203753FC8D20E7D057F07121D83D259
:1009510018D205752CC8D290301118E5484547606A
:100961000AE5481548700C15478008C211D221D2FA
:10097100B6D2C4301343E549603F301A17E54660EB
:100981000415468034C21A85554A85538B85518D8D
:10099100D28E8025E54A6004154A801DC28FC28E21
:1009A100D2C31549E5496007854F46D21A800AC26C
:1009B10013D220756907756AD0300714E5314530C7
:1009C100600AE5311531700815308004D2A4C207E0
:1009D100300D12E53C453B600AE53C153C700615BF
:1009E1003B8002C20D30190BE5546004155480039D
:1009F10075543C30060BE52A6004152A8003752ADC
:100A0100C8300312E5264525600AE526152670063D
:100A110015258002C203300E0AE53F6004153F80B0
:100A210002C20E30090FE535600415358007C20991
:100A3100D20175271430010DE527600415278005C3
:100A4100D20875271430050CE52C6004152C8004A0
:0F0A5100C205C290D0D0D082D083D0F0D0E03296
:03001B00021DFBC8
:091DFB0085538B85518DB2C33272
:03000300020006F2
:05000600C2A8D2A832DF
:0300130002000EDA
:05000E00C2AAD2AA32D3
:0300230002146C58
:10146C00C0E0C0D075D018309852C298E55E6003C9
:10147C0002150EE56614601B14602F1460332403F0
:10148C00600302150EE599B4AA0785995805668084
:10149C00718024E599C39404400EE599D3941150BE
:1014AC00078599590566805A800D85995A0566807D
:1014BC005185995B755E017566008046309943C213
:1014CC0099E557C39404503A000000000000000056
:1014DC000000000000000000000000000000000000
:1014EC0000000000000000000000000000000000F0
:1014FC00000000000000000074612557F8E6F59923
:07150C000557D0D0D0E032FA
:10120B00C10F012800013300013400C10401380073
:10121B00013900013A00013D00013E00012B00C1E4
:10122B000AC10B012900014200013201C10901353C
:10123B0000C101012700C108C102C1070230000033
:10124B00012A00C106C10302250000C10E013F00A7
:10125B00C10D023B0000C10CC10002360000C105EC
:03126B00012C0053
:071E16008E4C8F4DD2172204
:10193C00E4FEEF640170442080047E04803D20812D
:10194C00047E0180362082047E02802F2083047E58
:10195C000380282084047E0580212092047E098047
:10196C001A2094047E0A80132095047E07800C2094
:10197C0096047E0680052097027E08BF020C208606
:0C198C00047E0B800520C6027E0CAF0616
:01199800222C
:10102F00300F030211177F0112193C8F2D30220749
:10103F007F0212193C8F2E20041AD204852D3830CE
:10104F002203852E39201E03301F03852F3A752862
:10105F0014D20F22C204E538652D706D852D29E558
:10106F0029700EF533C209F535C201F527C2088084
:10107F0058E52965336015E529F46010C209E4F5D8
:10108F0035C201F527C2088529338030E52965333C
:10109F007037E529F46032E52964066017E52964A5
:1010AF00076011E5296408600BE52964096005E50F
:1010BF0029B40A1530010A30080FC208121118801E
:1010CF00082009057535C8D209E539652E70393004
:1010DF002236E52E640B6010E52E640C600AC20AFE
:1010EF00C20BC21BC21C8017E52EB40B06D20AC25C
:1010FF0014800CE52EB40C07301D04D20BC2142043
:09110F000306200703120C542210
:071E1D00D2A0C2A1D2A22253
:071E2400D2A0D2A1C2A2224C
:071E2B00D2A0C2A1D2A22245
:071E3200C2A0D2A1D2A2223E
:071E3900D2A0D2A1D2A22227
:1017D800302269E54E6401702C301E1730A108D202
:1017E80085C2A1D2A0800CC2A0C285D2A1D20C7F92
:1017F800198004C20C7F17121C1B300C047D038057
:10180800347D018030E54E64027038301F1730A1F6
:1018180008D287C2A1D2A2800CC2A2C287D2A1D20A
:101828000C7F198004C20C7F17121C1B300C047D1E
:101838000480027D027F03121D838007D20C7F176C
:10184800121C1B752501752690D203753FC8D20E50
:01185800226D
:101C40007D037F07121D83E4F51175C13F121E0449
:101C50000511E511C3946440F17D057F07021D83E2
:101C60007D057F07121D83E4F51175C13F121E0427
:091C70000511E511C3941540F1C2
:011C79002248
:1016CE008F10E510B41407754E147F138011E510BA
:1016DE00B41507754E157F158005754E067F0B12D6
:1016EE001C1B121C60C210C2C2C29175440075450B
:1016FE0096D210754C2E754DE0E510B40604D21737
:10170E008002C217302227E510B41407C285121EBC
:10171E00328013E510B41507C287121E248007C24B
:10172E0085D287121E2B752501752690D203E510E2
:10173E00B414047D03800BE510B415047D048002FF
:08174E007D027F03121D8322BE
:101B6600E4F54E7F11121C1BC217C202C210C20638
:101B7600C2A6D2C5D2C1201302D2B630220FC28568
:101B8600C287121E39752501752690D203C2C2C2BC
:091B960091753FC8D20E021C40FB
:10175600E54E24FE601624FD603A14603724FA60D4
:101766004824F8602F14602C24147065200C62E560
:101776004EB40105754E038003754E047F05121C99
:101786001B752AC8C219D206C211121D9430223204
:10179600D2C4802E20023A752AC8C219D206D2A611
:1017A600C2C5C2C1C2B6D20222752AC8C219D206A1
:1017B600754E0D7F05121C1BC211121D943022029C
:1017C600D2C4D2A6C2C5C2C1C2B67FC07E5D121E39
:0217D6001622D9
:10151300E54E121BF5153D0015AC0115AC02157A0D
:1015230005159F06153D07153D08158F1415A915BB
:10153300153D16153D17000015AF754E057F0912B1
:101543001C1B7D017F03121D83C2C5C2C1C210C211
:10155300C2C291754400754596D2107FE07E2E126B
:101563001E1630220FC287D285121E1D75250175E6
:101573002690D203021E1D301E047F148023301DCB
:10158300047F06801C301F1E7F158015301D047FCD
:1015930006800E301F047F158007800A301F057FE9
:0D15A300150216CE8000021B661217D8221A
:1012CC0020070320220C300D0302139C3022030252
:1012DC00139CE54E64016054E54E6402604EE54E8D
:1012EC0064036048E54E64046042E54E6405603C6E
:1012FC00E54E64066036E54E640B6030E54E640CDA
:10130C00602AE54E640D6024E54E640E601EE54EC9
:10131C00640F6018E54E64116012E54E6412600CA7
:10132C00E54E64146006E54E64157056C217C20291
:10133C00C219302207C212C216E4F534E4F54E7F0E
:10134C0011121C1BC211C206C210C2C2C291D2C45D
:10135C00121D94C2A6D2C5D2C1201302D2B630221D
:10136C0007C287C285121E39121E397525017526D2
:10137C0090D203753FC8D20ED205752CC8D29002FC
:10138C001C40E54E6003B413077D017F09121D83D9
:01139C00222E
:1018DA00E54E1424FA50028058C211121D947F0753
:1018EA00121C1B302237200748E54E6401601DE5B3
:1018FA004E64036017E54E64056011E54E640260AC
:10190A000BE54E64046005E54EB40602C2A4E53256
:10191A0075F0C8A485F030F531D207800DE532752F
:10192A00F0D2A485F03BF53CD20D7FA07E0F121EAB
:02193A00162273
:10185900E54E7023200311752AC8C219D206754EA8
:101869000B7F0D121C1B80617515567516667B144E
:101879007D0C7F03021AC4E54EB40B15C206E4F5CC
:101889004E7F11121C1BC217D203752501752690B4
:1018990022E54E64036006E54E6404703320073088
:1018A900C206E54EB40307754E0E7F018005754EDD
:1018B9000F7F03121C1BD2C5D2C1C2A6201302D2AC
:1018C900B6C217C210C2C2C2917FE07E2E121E1686
:0118D90022EC
:10199900E54EB413067D017F07803FE54E701D7546
:1019A9004E137D017F07121D83C2B6754001754133
:1019B900F4D214754400754596D21022E54E64059B
:1019C9006011E54E6406600BE54E64146005E54E52
:0E19D900B4150A754E137D207F02121D832265
:101BCE00EF14601114601514601624037018C2B25D
:101BDE00C2B4D2B522C2B2D2B4C2B522D2B280023F
:071BEE00C2B2C2B4C2B5226D
:101AF300EF4E6010E543C394035004054380137510
:101B03004303800EE543D39400400415438003E46C
:101B1300F543AF43121BCEE4FFFE121CED7F0A1206
:0A1B23001CD9AD43E4FFFE021CC311
:10111800E529640B6025E529640C601F30250F75EF
:1011280015567516667B147D147F01121AC42000AB
:1011380004D200D2A37536077537D030140DE54EAA
:10114800B413087540017541F48002C214E52914EE
:10115800B40D0040030211F390116E75F003A4C59D
:101168008325F0C583730211950211A70211AA0203
:1011780011AD0211B00211B30211B60211CC021165
:10118800E50211EB0211F30211F30211F1200E5BDB
:10119800302203300706202252200D4F0215130279
:1011A80017560218DA0218590212CC02199920228D
:1011B8000F202237E54E64016031E54E6402602B52
:1011C8007D04801420220F202221E54E6401601B3B
:1011D800E54E640260157D057F07021D837F017E51
:0C11E800008003E4FFFE021AF3C2C222E2
:04126E00C122C123B5
:1019E70075935F7594A0C285C2877591FC75920245
:1019F700C290C291E4F595759610D2A7D2A4121E93
:101A070039D2A3C2A6C2A575B30375B303D2B3D2A5
:101A1700B675B34075B40475BB70C2C2C2C0D2C537
:0A1A2700D2C1E4F5C9F5CAD2C42209
:101D150053877F759850438E04759CEE438E01431F
:031D25008E1022FB
:101D4E00438E805389F0438901758A9A758CA9C296
:021D5E008D22D4
:101D6000438E4053890F438910758B9A758DA9C294
:021D70008F22C0
:031D280075C13F43
:101D2B00121E04E55E60087F01120A60E4F55E2274
:100E1500D224E4F511302405121D2880F8D224E4EB
:100E2500F511302405121D2880F8D224E4F511307F
:100E3500240875C13F121D2B80F5D224E4F511302D
:100E45002405121D2B80F8D224E4F5113024051257
:100E55001D2B80F8D224E4F51130240875C13F120A
:100E65001D2B80F5D224E4F511302405121D2B80AD
:100E7500F8D224E4F51130240875C13F121D2B80EA
:100E8500F5D224E4F51130241575C13F0511E5119E
:100E9500C394C84004D225C224121D2B80E8E4F572
:100EA5001075C13F121E040510E510C3941540F1DD
:100EB500E56DC394014007E56DD394114003756D4D
:100EC50001E56EC394014007E56ED3940B401A7596
:100ED5006E02AF6E121D01E4F51075C13F121E04BE
:100EE5000510E510C3941540F1E54BC39405400783
:100EF500E54BD3941E4003754B0AE532C39401407C
:100F050007E532D3940A40037532017515567516F7
:0C0F1500667B147D287F01121AC4C2A361
:010F210022AD
:101D3B00E4F51075C13F121E040510E510C394FAAB
:021D4B0040F165
:011D4D002273
:10139D00C2AF121D4E121D60121D15D2ACC2B9D2B4
:1013AD00A9D2AB75C13F1219E7C2A5121D3BD2A53B
:1013BD00D28CD2AF120E15E4FFFE121CAC8F43E59A
:1013CD0043C394004007E543D394034003754301A1
:1013DD00AF43121BCEE55D64027032C2C2C291C230
:1013ED00AF755D03C2A5121D3BD2A5121D3B121D8B
:1013FD003BE55DB40315E4F55D7515567516667B15
:10140D00147D287F01121AC4E4F54ED2AF75C13F89
:10141D00E54E700B201308202005D2B6121E393070
:10142D0018147F11121C1BC210C2C2C2917D037F02
:10143D0007121D83C218302105C221121D941210EE
:10144D002FE55E6008E4FF120A60E4F55E20158565
:0F145D003022061200260213E21204400213E2AC
:10127200014E00C11BC11C02470000C111C112C1B5
:1012820016014900014A00C113C11A014600014F6B
:1012920000015500C11DC11EC11FC115024C000035
:1012A200C117C119015400C118C110024400000144
:0212B2004B00EF
:041C7A007F017E0068
:101C7E00D3EF9400EE9400400B7D64DDFEEF1F70F9
:041C8E00EF1E80ECD9
:011C9200222F
:0B1DCD000000007F417E88DEFEDFFC8E
:011DD80022E8
:0A1DE50000007F577E0CDEFEDFFCDD
:011DEF0022D1
:0D1DB200007F027E187DAFDDFEDEFCDFFA53
:011DBF002201
:0E1DA30000007F067E0B7DEBDDFEDEFCDFFA2E
:011DB100220F
:101D72008F15E515D394004007121E0D151580F23C
:011D8200223E
:081E04007F6C7E91DEFEDFFC25
:011E0C0022B3
:081E0D007F057E4ADEFEDFFCCA
:011E150022AA
:0B1DD9000000007F0D7EE5DEFEDFFC59
:011DE40022DC
:0A1DF00000007F167E80DEFEDFFC9F
:011DFA0022C6
:021C1B00AD0713
:101C1D00D215C2A7121E04D2A7121DF0E4FCECC30C
:101C2D009D500DC2A7121E0DD2A7121DD90C80EE0C
:021C3D00C215CE
:011C3F002282
:100F2200E4FBFAF9FCC22630B30302102C7F04FE64
:100F3200121C7E30B303021029D22630262520B39C
:100F420014121C7A0BBB00010AD3EB945EEA9401E3
:100F520040EC7F00227F027E00121C7E30B3DCC296
:100F62002680D8C3EB9464EA940050037F0022E405
:100F7200FAFBD22630262530B314121C7A0BBB00A2
:100F8200010AD3EB9450EA940040EC7F00227F02E6
:100F92007E00121C7E20B3DCC22680D8C3EB940AEA
:100FA200EA940050037F0022E4FCE4FAFBD22630EC
:100FB200262520B314121C7A0BBB00010AD3EB9432
:100FC20014EA940040EC7F00227F027E00121C7E15
:100FD20030B3DCC22680D8C3EB9402EA94005003FB
:100FE2007F0022E4FAFBD22630262630B315121CEB
:100FF2007A0BBB00010AD3EB9432EA940040ECE98D
:1010020004FF227F027E00121C7E20B3DBC22680F8
:10101200D7C3EB940AEA940050037F0022090CEC38
:0C102200641B70867F00227F00227F008C
:01102E00229F
:0E1B9F00C291C206C219C202C2A6D2C5D2C1EC
:101BAD00C211C221AF6D121A31C2B6E54B75F0C824
:101BBD00A485F047F548D211C2127D037F07021D9F
:011BCD008394
:10002600C2AF120F22D2AFEF121BF50056010056D7
:100036000300A805012B07019509020A0B03D90D38
:1000460003FE11029613033115043C170000043F0A
:10005600E54E6409601BE54E640A6015E54E640EC4
:10006600600FE54E640F6009E54E641060030204FC
:100076003FBF0107754E017D018005754E027D0269
:100086007F03121D83C210C2C2121B9F75440075E6
:100096004596D210754C2E754DE0D217753FC8D2D5
:1000A6000E22E54E24FE601524F7603A14604B24B8
:1000B600FE605314605C240E600302043FE54EB4F8
:1000C6000105754E098003754E0AC211121D94D2A0
:1000D600C4D2C5D2C1C2A6D2B6C210C2C2C291751E
:1000E600543CD2198036754E0DC211121D94D2C4DD
:1000F600D2A6C2C5C2C1C2B68022754E10C21112A6
:100106001D94D2B68016754E0975543CD219D2B6D6
:10011600800A754E0A75543CD219D2B6754C75755F
:100126004D30D21722C211121D9430070302043F2C
:10013600E54E64016041E54E6403603BE54E6405AF
:100146006035E54E6407602FE54E64096029E54E8B
:10015600640E6023E54E6402601DE54E640460177C
:10016600E54E64066011E54E6408600BE54E640AD0
:100176006005E54EB40F02C2A4E53275F0C8A48549
:10018600F030F531D207754C2E754DE0D21722E5C9
:100196004E6004641370167D037F07121D83E54EBF
:1001A600B41302D2B6C210C2C2C2918038E54E6400
:1001B60014600BE54E64066005E54EB415167D0128
:1001C6007F03121D83C217C287D285121E1D754E6C
:1001D60005020279E54E6416600BE54E640860057B
:1001E600E54EB4170D754E07C287D285121E1D0245
:1001F6000279E54E64056009E54E64076003020472
:100206003F0203F5201D030203D6E54E6416600B7C
:10021600E54E64076005E54EB4170C754E08C285B9
:10022600D287121E2B804CE54E6414600BE54E649B
:10023600056005E54EB415157D027F03121D83C2C8
:1002460085D287121E2BC217754E068026E54E6094
:1002560004641370297D037F07121D83E54EB413D2
:1002660002D2B6C210C2C2C291754E08D287C285EA
:10027600121E2B754C5D754DC0D2170203B8E54EA4
:1002860064066009E54E6408600302043F0203F554
:10029600E54E6004641370297D037F07121D83E514
:1002A6004EB41302D2B6C210C2C2C291754E16C265
:1002B60087C285121E32754C5D754DC0C21702038A
:1002C600B8E54E6405600BE54E64066005E54EB480
:1002D600151E7D037F03121D83C217C287C28512B6
:1002E6001E32754E14754C5D754DC0C2170203B8AB
:1002F600E54E6407600BE54E64086005E54EB417ED
:1003060015754E16C287C285121E32754C5D754D27
:10031600C0C2170203B8E54E641470030203CDE5AC
:100326004E6416600302043F0203CD201D03020340
:10033600D6E54E6408600BE54E64076005E54EB4ED
:100346001614754E17C285C287121E24754C5D752C
:100356004DC0C217805CE54E6414600BE54E640523
:100366006005E54EB4061D7D047F03121D83C2851C
:10037600C287121E24C217754E15754C5D754DC089
:10038600C217802EE54E60046413702F7D037F072D
:10039600121D83E54EB41302D2B6C210C2C2C29178
:1003A600754E17C287C285121E24754C5D754DC0E9
:1003B600C217752501752690D20322E54E64156095
:1003C60006E54E64177072754C5D754DC0C21722F6
:1003D600021B66E54E60046413705E7D037F0712A0
:1003E6001D83E54EB41302D2B6754E0C121BAD75C5
:1003F6004C5D754DC0D21722C217C202C219E4F570
:100406004EC211C206C210C2C2C291D2C4121D94FB
:10041600C2A6D2C5D2C1D2B6C287C285121E39754E
:100426002501752690D203753FC8D20ED205752CCC
:09043600C8D290021C401217D834
:01043F00229A
:0C1AB8007515567516667B147D0C7F03B7
:101AC400AC07C2B6E516F404755200F553C3E495A9
:101AD40016E49515755000F55185538B85518DD2BB
:0F1AE4008E8C498D558B4F85554AC21AD21322CD
:1015B000E54EB41302D2B6D216302617754E02C2CB
:1015C00010C2C2C291D287121E2B7F03121C1B7D38
:1015D000028015754E01C210C2C2C291D285121E80
:1015E0001D7F01121C1B7D017F03121D83121BAD89
:1015F000C2C5C2C1C2C4C20C754400754596D210A2
:10160000754C2E754DE0D217752501752690D203C5
:10161000753FC8D20EE4FD75C13F121E040DBDDC3E
:10162000F6E4FD75C13F121E040DBDB4F67D047FC6
:1016300007121D83200004D200D2A3753607753728
:01164000D0D9
:011641002286
:100C5400200A03020D34301B03020D34D21BE54E6F
:100C6400B418004003020D34900C73F82828730262
:100C74000CBB020CC2020D34020D34020CD5020C62
:100C8400E1020CE1020CE1020CE1020D34020D2B35
:100C9400020CE1020CE1020CE1020D2F020D340200
:100CA4000CE1020CBB020CBB020CBB020CE1020CFB
:100CB400E1020CE1020CE1C2261215B0807220118F
:100CC4006F7F01121C1B121BADC2C5C2C1C2C480FE
:100CD4005F121AB87D017F08121D838053754E017F
:100CE4007F01121C1B7D017F03121D83C202C206F9
:100CF400C2A6C210C2C2C291C287D285121E1D12E0
:100D04001BADC2C5C2C1C2C4754400754596D2109C
:100D1400754C2E754DE0D217752501752690D203BA
:100D2400753FC8D20E80097F0F80027F01121C1B01
:100D3400200B03020E14301C03020E14201D0302A8
:100D44000E14D21CE54EB418004003020E14900D8C
:100D540059F8282873020DA1020E14020DA6020DE3
:100D6400B8020E14020DC2020DC2020DC2020DC25F
:100D7400020E0B020E14020DC2020DC2020DC202BB
:100D84000E14020E0F020DC2020DA1020DA1020DDE
:100D9400A1020DC2020DC2020DC2020DC2D2260270
:100DA40015B020116B7F03121C1B121BADC2C5C2F0
:100DB400C1C2C422121AB87D027F08021D83754E77
:100DC400027F03121C1B7D027F03121D83C202C219
:100DD40006C2A6C210C2C2C291C285D287121E2BFD
:100DE400121BADC2C5C2C1C2C4754400754596D2BA
:100DF40010754C2E754DE0D217752501752690D2CD
:100E040003753FC8D20E227F0F80027F03121C1B82
:010E140022BB
:10044000C2AF120F228F10D2AFE510121BF5047944
:1004500001047903055F0505E20705FD0906610B47
:10046000078C0D07B40F07D81106C5130729150807
:100470000F1708281900000840121E1DE54EB41879
:1004800000400302084090048DF82828730204D528
:1004900002051E02052F0205410205500204D50285
:1004A00004D50204D50204D50204D50204D5020401
:1004B000D50204D50204D50204D50204D50204D520
:1004C0000208400208400204D50204D50204D50205
:1004D00004D50204D5E510B40107754E017D0180F5
:1004E00005754E027D027F03121D83E54EB4130293
:1004F000D2B6C210C2C2200004D200D2A375360701
:100500007537D0121B9FC20C754400754596D210EA
:10051000754C2E754DE0D217753FC8D20E223011A2
:1005200003020840E51064016003020840800F30B8
:100530001103020840E51064036003020840021B37
:10054000ADE51064036003020840121AB80207D137
:10055000E51064016003020840121AB80207C7E5FB
:100560004E24FE601524F7603A14604B24FE60535D
:1005700014605C240E6003020840E54EB40105756A
:100580004E098003754E0AC211121D94D2C4D2C501
:10059000D2C1C2A6D2B6C210C2C2C29175543CD258
:1005A000198036754E0DC211121D94D2C4D2A6C246
:1005B000C5C2C1C2B68022754E10C211121D94D29E
:1005C000B68016754E0975543CD219D2B6800A759C
:1005D0004E0A75543CD219D2B6754C75754D30D251
:1005E0001722C211121D94E53275F0D2A485F03B9A
:1005F000F53CD20D754C2E754DE0D21722E54E60BC
:1006000003B413167D037F07121D83E54EB4130256
:10061000D2B6C210C2C2C2918031E54E6414600BE2
:10062000E54E64066005E54EB4150F7D017F0312AB
:100630001D83C217754E050206C3E54E6416600B96
:10064000E54E64086005E54EB41705754E078073E6
:10065000E54E64056009E54E6407600302084080CA
:1006600062E54E64166048E54E64076042E54EB4AC
:100670001702803BE54E6414600BE54E640560058F
:10068000E54EB4150F7D027F03121D83C217754E10
:1006900006020727E54E6003B413197D037F071296
:1006A0001D83E54EB41302D2B6C210C2C2C2917508
:1006B0004E088073E54E64066009E54E64086003E9
:1006C0000208408062E54E6003B413167D037F0785
:1006D000121D83E54EB41302D2B6C210C2C2C2913B
:1006E0008031E54E6405600BE54E64066005E54E1D
:1006F000B4150F7D037F03121D83C217754E1402BC
:10070000078AE54E6407600BE54E64086005E54E18
:10071000B41705754E168072E54E64146009E54EF7
:10072000641660030208408061E54E64086047E596
:100730004E64076041E54EB41602803AE54E6414FB
:10074000600BE54E64056005E54EB4060E7D047F42
:1007500003121D83C217754E158050E54E6003B419
:1007600013197D037F07121D83E54EB41302D2B621
:10077000C210C2C2C291754E178030E54E6415603A
:1007800009E54E64176003020840801FE54E6007CC
:10079000641360030208407D037F07121D83E54E4A
:1007A000B41302D2B6754E0C121BAD754C5D754D6F
:1007B000C0D21722E54E64036005E54EB40403126F
:1007C0001AB8E54EB403047D028008E54E64047057
:1007D0006F7D017F08021D83C217C202C219E4F5B2
:1007E0004EC211C206C210C2C2C291D2C4121D941E
:1007F000C2A6D2C5D2C1D2B6752501752690D20344
:10080000753FC8D20ED205752CC8D290021C40C2CA
:100810000CE54EB401047D018007E54EB402077D6E
:10082000027F03121D838015E54EB401047D038011
:1008300007E54EB402077D047F03121D83121E1DBF
:010840002295
:1012B400015E00016600015700C124025F000001C5
:0712C4005D00015600C1A509
:101D83007561AA8F628D63EF2DF564E4F557D299DF
:011D9300222D
:101C9300C226E559255AFFE433FE7C00EFB55B0607
:081CA300ECB50602D226A226D0
:011CAB002216
:100A6000AD07121C934003020C53E55864AA6003BF
:100A7000020C53E55924FCB40E004003020C5390C1
:100A80000A8D75F003A4C58325F0C58373020AB7E8
:100A9000020ADD020AFC020B16020B30020B4602B0
:100AA0000B5C020B72020B88020BF8020C18020C92
:100AB00026020C3A020C3DE55AC394015003020C85
:100AC00053E55AD394104003020C53855A6DED70D0
:100AD00009E55D7005AF6D121A31C22422E55AC3D3
:100AE00094015003020C53E55AD394084003020CBE
:100AF00053855A6EAF6E121D01C22422E55AC3946B
:100B0000005003020C53E55AD3943C4003020C53AB
:100B1000855A4BC22422E55AC394015003020C5358
:100B2000E55AD3940A4003020C53855A32C2242258
:100B3000E55AB40105D222C22422E55A6003020C10
:100B400053C222C22422E55AB40105D21DC2242276
:100B5000E55A6003020C53C21DC22422E55AB401B7
:100B600005D21EC22422E55A6003020C53C21EC2E3
:100B70002422E55AB40105D21FC22422E55A60039B
:100B8000020C53C21FC22422E55A704DE54E641375
:100B90006003020C53C214C217C202C219C212C2AD
:100BA00016F534F54E7F11121C1BC211C206C2107D
:100BB000C2C2C291D2C4121D94C2A6D2C5D2C12053
:100BC0001302D2B6C287C285121E39752501752659
:100BD00090D203753FC8D20E22E55A64017074E5C5
:100BE0004E7070754E13D2147540017541F4C2B643
:100BF000F544754596D21022E55AD394004016E587
:100C00005A940B5010AF5A121D01202346AF6D129B
:100C10001A31021E04021D94E55A7037755F06757D
:100C20006040755D0122E55A7005F556C22422E543
:100C30005AB4011F755601C22422C22422E55AC3A8
:100C40009400400FE55AD394015008E55A24FF92CE
:040C500025C2242273
:10164E0002139DE493A3F8E493A34003F68001F202
:10165E0008DFF48029E493A3F85407240CC8C3339D
:10166E00C4540F4420C8834004F456800146F6DF6C
:10167E00E4800B01020408102040809011F4E47EF7
:10168E00019360BCA3FF543F30E509541FFEE49361
:10169E00A360010ECF54C025E060A840B8E493A328
:1016AE00FAE493A3F8E493A3C8C582C8CAC583CA53
:1016BE00F0A3C8C582C8CAC583CADFE9DEE780BE0B
:0112CB000022
:101BF500D083D082F8E4937012740193700DA3A37F
:101C050093F8740193F5828883E473740293686092
:061C1500EFA3A3A380DF92
:00000001FF
